:1000000002038E20312DC0D0022803C0D0202E1034
:1000100002280B20122BC0D0022813C0D0022300CC
:10002000021BC7C0D0201F1C022823C0D002282BCF
:10003000021C04202608C29630B2FDD29632022855
:1000400040D216320228501A3A13DF1159114F04C8
:10005000B5071006F506D715E01532134D19F2163F
:100060005319C716FB16E416EE15D0161D162B16DF
:100070003016241617160115B7158C15C016F81270
:10008000F2137712F8146115E1152C138E14A315D1
:10009000EC15F616DE1637170F19BA19CD115518CB
:1000A000DA19D6171F17231727172D1733173717E6
:1000B0003B173F17431747174B10B118E917521852
:1000C0003112100E941027103107DF0864010F0E53
:1000D0000A080A080305040C0606060606060F0FA2
:1000E0000F0F0F0F0F0F0F0F0F0F0F0F53746F70B6
:1000F0002254727920616761696E22526561647968
:1001000022202D20696E206C696E65202208641102
:10011000B20BC806891AF8047B1A251A320547045F
:1001200074067D09E406C00B1B0B5B19270D291B08
:10013000F11BF70B240D2D0FA90E900626199D1B00
:10014000DD0D2B08C30F9A16630BD010680CBA1084
:100150005D0C3E16590E060F2E0CD3104A0BD20B17
:10016000300BFB0AD20BBA0BC01A3A1B15116111E6
:1001700066051A0812804C455481434C4541528211
:100180005055534883474F544F8450574D855048DE
:10019000302E86554987554F88504F5089505249C7
:1001A0004E5489502E893F8A43414C4C8B44494DD3
:1001B0008C535452494E478D424155448E434C4FC7
:1001C000434B8F5048312E9053544F50914F4E54C3
:1001D000494D45924F4E45583193524554499444A8
:1001E0004F95524553544F52459652454D974E4563
:1001F0005854984F4E455252994F4E9A494E505529
:10020000549B524541449C444154419D5245545550
:10021000524E9E49469F474F535542A0464F52A1CA
:100220005748494C45A2554E54494CA3454E44A409
:10023000544142A55448454EA6544FA753544550E7
:10024000A8454C5345A9535043AA4352AB49444C8B
:1002500045AC535440AD4C4440AE50474DAF525264
:100260004F4DE028E12A2AE22AE32BE42FE52DE690
:100270002E584F522EE72E414E442EE82E4F522E2E
:10028000EA3DEB3E3DEC3C3DED3C3EEE3CEF3EB00E
:10029000414253B1494E54B253474EB34E4F54B4FA
:1002A000434F53B554414EB653494EB7535152B8CC
:1002B000434259B9455850BA41544EBB4C4F47BCC4
:1002C000444259BD584259BE5049BF524E44C0479E
:1002D0004554C146524545C24C454EC35854414C05
:1002E000C44D544F50C64945C74950C854494D455F
:1002F0005230C954494D455231CA504F525433C5FA
:1003000054494D45CB504F525432CC54434F4ECDAF
:10031000544D4F44CE504F525430CF504F52543121
:10032000D050434F4ED141534328D25553494E47A5
:1003300028D2552E28D343485228F052554EF14C1E
:10034000495354F24E554C4CF34E4557F4434F4EDF
:1003500054F550524F47F658464552F752414DF822
:10036000524F4DF94650524F47FA4552415345FFBF
:1003700045787472612069676E6F72656422412DE1
:10038000737461636B22432D737461636B2275C751
:10039000AA75C75575878075985A758920758854D0
:1003A000758DFA902801E493B4AA03122890787FFF
:1003B000E4F6D8FD753E4D853E81751360751411C8
:1003C000906000E0C39431F545C2E2FFA31205CA74
:1003D0001208EFA31205CA90305FE0903000B4A578
:1003E00008E545C2E06404602DBF02028003BF033C
:1003F000051206AE8017AB83A982A3E58364606013
:100400000C745AF0E0B45A05E4F0BBE0E990310A0C
:1004100012061C1206891206A01218E3E545B4055F
:1004200003122839500D30E024906010E0B4551DBF
:10043000020864E4FBF978048013D8FE12180178EE
:100440000230B0F620B0FD30B0FD1208EF90235B13
:100450001206E1021A327F007E017A5F78FF1204F1
:10046000BA0EE5CB1204BAE5CA7E0379097B3112D4
:1004700004BA803C90312AD2338005903128C233AF
:1004800012058FC29512103E70CC7CFED21D120553
:1004900066121B0EECF4121717121C871205251298
:1004A00006D7A80EAA0F74550EBE00010F1204BD88
:1004B000D29502054C8B7F121C451217E57D01FC7D
:1004C0001204FF12050B20330C6C70251218D27029
:1004D000E453D0E7226C7014EC1204FF12050412EE
:1004E0000504120504DDF512050B80DD0DECBD19C8
:1004F000CED29575D000302FDB902322021B498A83
:100500007F121C5400000000000022D294121C36FE
:10051000D29322750F0CD50FFD22C29575D01812FB
:1005200004B5D29522120597A3AB13A914C3E58293
:1005300099FEE5839BFF22120536C28E85408D858C
:10054000418BC28FD28E22C21712054F02120112A6
:1005500010A0AC0050027C01120566BC0011A385FE
:10056000831385821422906010E0B4550ADC0122C6
:10057000A31205BCA380F2101DF59023510204FCC8
:10058000E0FAA3E0F822CBC583CBC9C582C922E03B
:10059000F540A3E0F54122D229120FEA120B556073
:1005A00015A320290C1205DD1205D3E0202A0740EF
:1005B000051205F080E6C22922903300D22980DCA2
:1005C000E0C0E0A3E0F582D08322E0FBA3E0F922C3
:1005D0001205D3C5827002158314C58222C22AE097
:1005E000B5030BA3E01205D3B50103B3B22AB322BE
:1005F0002582F58250020583221206CB1205B974BA
:10060000061205F012058690310812061F1205CA5F
:100610009031221205C0120A9190310412061FEB8C
:10062000F0A3E9F0A322120FCF90312212061F0E81
:100630008E3F0206919031041205C01205D0E06091
:1006400020A3B5070FE0B5060BE5829402F8E58319
:100650009400FA22E582C39409F58250E115838063
:10066000DD120F28C3120649E89406F9EA9400FB4C
:1006700090310612061F1205DD4042D32290600021
:10068000E4F0A3E58330E7F8229033007401F0C270
:10069000151205F990310A1205CA1205B91206AEF3
:1006A0009000FEE4F07511FE7509FEC21722A3E466
:1006B000F0E07009EBB583F6E9B582F22202182B5F
:1006C00012103E50CC121034B449D5301202C2AAD6
:1006D000532220321206D77D0D1207557D0A0207DC
:1006E000551206D7E493C2E7B4220122D234FD1298
:1006F0000755A380051205867C0D1034E7E06003E2
:10070000B5040122B40DE7021B3FB4041E1206D744
:10071000757F3078071207DFFDB40802747FB47F5D
:10072000E9B8071C7D0712075580EA121C54B40D66
:10073000030206D7B4200040ED08B856E91880E45B
:10074000187D081207551207537D0880D97E0000D6
:100750005067417D20C0E0C083C08230350512075C
:10076000DA80F8ED302C061228400207B2301C0661
:100770001228300207B230270930190612283C022D
:1007800007B2301B2690312412058FC2971205370D
:10079000EDD37D0913308FFD9297120537DDF530CB
:1007A0008FFD120537308FFDFD80073099FDC2990E
:1007B0008D99BD0D03751600BD0A0CE51560087D09
:1007C000001207551470F8BD08021516BD20004030
:1007D000020516D082D083D0E02212081B5032309E
:1007E00032051228608011301E051228338009302E
:1007F00098FDE599C298C2E7B41302D235B411024C
:10080000C235B4030430302822C228B41702D228DB
:10081000D322D21D12054F101D4A22303203022866
:1008200068301E03022836A2982290235B1206E449
:10083000C235120D331206D71028EF202F030208FD
:10084000CC02054CE548A949B548F9C9954CE9954C
:100850004B221208444045D214C210A211922B9090
:100860003126804112068F120CBD120B55605112B9
:10087000100E12108D120D3FC22F853E81202F06C3
:10088000850A428508431207DA202F26B018500641
:10089000903100F0D2182014192010B63016132011
:1008A00011109031207C02120C06D2111205800228
:1008B0000BB412096612107F50C0302F03021A5079
:1008C000021A3A12107F850A42850843D217900017
:1008D000ECD220021B69B4C8058B8C898A22B4C96A
:1008E000058B8D898B22B4CA0389B022B4CE0389CB
:1008F0008022120A5DB4CB0389A022B4C60389A862
:1009000022B4C70389B822B4CC03898822B4CD03AA
:10091000898922B4CF32899022F50F121034120A3D
:100920004FE50FB4C3030218E9120FDDE50FB4C49D
:100930000990310A12061F020691B4C599A2AFC2EE
:10094000AF8B48894992AF22B4D062898722B4D153
:10095000C8121024B42456120AAD120EE212171A4D
:10096000120A67020994121027302D0FB42000508C
:100970000A122870121034540F8057B4C30050CE9E
:1009800030E761B4BC08120A61120A5DF722B4BDF7
:1009900009120A618B7F121C6322B4AB004009B4B8
:1009A000B000500924F9801DB4A4004003021B3F8D
:1009B000302F12B49000400DB4A0028008B497020A
:1009C0008003B496E8121034900123B4800280961C
:1009D000543F232582F582E493C0E0A3E493D083BF
:1009E000F582E473121015405DC2151205867FEA88
:1009F000120DFF121027B42214AF3F121034121040
:100A00003E60AAF0B4222B740DF0021034C083C0F3
:100A1000821210154097D000D002AF3F121808B4D0
:100A20000D0122DF08740D121C54020F911217E5FC
:100A300080EADF09120A07120F9102104AA380BB55
:100A4000901AE2020D09120A4C02114F121063C0F3
:100A500002C0007FEA1210AED001D00322BB00E03A
:100A600022121034120DF8120A4F121705EEBF00B1
:100A7000CF22120FE2120A5D09E960C490310485A9
:100A80003FF0120A9F90310A121826853F82758323
:100A900000C3E99582F9EB9583FB492275F00612B4
:100AA00005C0E9A42582F9E5F03583FB22120A721C
:100AB000C003C0017F2C120DFF120FDAE9B53F0011
:100AC0004003020A4019D0E029F9D00350010B027B
:100AD0000DFD120A4CC003C00112114F7FA6121067
:100AE000AE121027B4A7081210341210B1800312EE
:100AF000169274EF120C9A120CA67B30A9001211F8
:100B00004F12114F120FF1A801120C0BD008D00A8E
:100B10007C01120C0B12100E02087A1210B1121086
:100B20001E50F82212106312114C12101E50F522A2
:100B3000120B7DF9121027B4A503121034B9000D61
:100B40007FA812104C60E8121034B4A8F31210A061
:100B50005062020966E01420E73522120BAB121036
:100B60000E10250930150312068F0208781014069E
:100B70005322BD02087AA22B921102087A1210B1F8
:100B8000121416600274FF22120FEAE0FFDF0690D3
:100B9000233D020D0920E7F7A3E0B50208A31FE0FB
:100BA000B50002A322EF1205F080E012109A120B9A
:100BB0008802107F120B88020B5E120B7DF48003FB
:100BC000120B7D7C03FD800E12109A88150208C05E
:100BD000D2257C027D55120C24121C36F583081296
:100BE0001C36F58208E0B401030208C0ED70030270
:100BF0000B5E8811F46003020B5E22120BAB7C02C9
:100C0000120C06020B1574FD120C9A757F30E50864
:100C1000121C5418E50A121C5418EC121C542274AD
:100C200003120C9AA811757F30121C36B504020805
:100C3000227003020CABB401E6120C9880E67C0132
:100C4000120C24880F790B121C36F70908B90FF71C
:100C5000120E945004AA0BA80CEAB50B4EE8B50C82
:100C60004A121159740E250FF87A308A7F121C36F9
:100C700008C0E0121159C0001219F2121677AB0B1E
:100C8000A90C12114F7A30D000121159121C78D0D1
:100C9000E06001B372D5401974112511B4610040B0
:100CA0000AC51114F82212107F50FA900386020D23
:100CB00009850D0A850E0802087A120CC6120FEA81
:100CC00012100E12108DC50AC512C50AC508C5102E
:100CD000C50822120CC612101E401D1210B11210AF
:100CE00027B42C02800312107F120CC6121063125C
:100CF000114C12101E50DC22B49C0512103480DB03
:100D0000B40109120CC6902309021B4912104A12A1
:100D1000107F40EF80C0121027B42305D21B0210B1
:100D200024B440D3D219021024D236D237120D1671
:100D3000120D3A5323F553263F2212103E4008026B
:100D400006D712101E40F8120FF850F6B4A409127C
:100D50000FE2951640EC8006B4A90B120FE260E298
:100D60001207531480F8B4D318121024B4240812B4
:100D7000117A120FDD8006120FDA120DFDAD01801F
:100D800008B4AA0A1210347D0D12075580B4B4D2EB
:100D90005E121024B446187517F012102412103485
:100DA000540F6007B40300500274034217802FB43D
:100DB00030087517001210348024B42321120DE47A
:100DC0008F17B42E14121024120DE4EF251724F7F8
:100DD00050030209ADEFC44217E517C4F517120D11
:100DE000FD020D427F00B4230E0F12102480F71273
:100DF00010415003B4A841227FE01210AE7F2912A7
:100E00001031B507CD22120FDA121031B483061259
:100E10000E1E020B15B49FBA120E1E020BFEB90075
:100E20000912109A12104A020BAE7F2C12104CB409
:100E30002CA01912103480E612101540061206F587
:100E4000020D421210B17448B516005003120D3F46
:100E50003037161213B840111215B77009120FDD92
:100E6000121C93020D421215D0121C877401020D40
:100E70005E1210241223B1400CB45F0122B4410071
:100E80004004B45B00B32230D543901A13020D091D
:100E9000D2D58002C2D5121027120E7D500420D563
:100EA000E922FFE4FDFE120E714007CF2DCF7D1A1F
:100EB00080F3C215B4E032430680120635C002C08A
:100EC0000050C420D52B790A7B00120F04120FE5C5
:100ED000BB00B7D082D083E0149940AE1205D01287
:100EE0000A9CC9C8C9CBCACB2220D59E120635C3DD
:100EF00022120FE5BB0093D000D002120F04121093
:100F00001E508D2209E96082FC903108120A9CAFC4
:100F100083AE8290310612182690310812061F887F
:100F2000828A83ECF01205D0EFF0A3EEF022120FCC
:100F3000F812101E5008120D3F7D3F120755D222A5
:100F4000120710C222750F30750E071210154010CF
:100F5000120EE2AB0FA90E120A1A12101E50DA225C
:100F6000121B07121C1C701B121B0E121063121195
:100F70004C121B0712101E4013E0B42C06A3121BC8
:100F80000E80C89000F11206E1021AFEE0B40D01D5
:100F9000229003701206E1020D3F120FCF8B4B8996
:100FA0004C903126D210020F2812109ABA000AE88B
:100FB00020E70628904100F5821209E253D0E7228B
:100FC000120FDA12191C8B4089417F2C120DFF126F
:100FD00010B17F2C1210AE0217051210B11213DFE0
:100FE000E922121034120DF880F3851383851482E0
:100FF00022850A8385088222121027B422028003E8
:1010000002108B120FF1A37C221206FAA3C3858370
:101010000A85820822121027B42470020A72121064
:1010200027B42C67121034D2D38A7F121C36C2D355
:1010300022121027D2D308B800010AC2D3221210FC
:1010400027B40D02E422B43A42227F0D12103E5022
:10105000F8B507012212103480F212103412103E3B
:1010600070F822120E948035120CA67C03120C0626
:1010700002087AB43A03021034B4A87912105D124F
:101080001027B40DEE121024B40102D322C5082497
:1010900003C50810D70122050A221210A0405622CB
:1010A000120FF1121C8D12100E8A83888222120DEB
:1010B000FF7ACDC002C224E581240C5003021B46F6
:1010C000E509943850030213D3202417120E9450CC
:1010D0000F12116E500D121027B4E00774CE805C11
:1010E000121159121027B4E000500EB4B000503F56
:1010F000D0022024B8C3021B41541F202405B4058C
:1011000042740924CEFA90000093FCD0E0FD93B520
:101110000404B40C98D35095C005C00212103412C8
:1011200010B3D0E090005724321209D20210B71247
:101130001034242E2024BEB4EC0050E8C0E0120D80
:10114000F880DFB403AF1210340210B7120EE212AF
:1011500014160216CC7A3178131213C4D224021654
:10116000CC120FDA80E9120FDA120EE280EB1210C5
:1011700027B4D115121024B42406120AAD0215F9B1
:10118000121717121034020DFD120FF1121C1CB4AD
:10119000FF02D3227006C3D22402100E540B60F358
:1011A000901A0330E003901ABE30E103902311023D
:1011B0001B49120D1612160B1210A0E4FBF9401673
:1011C000121B0E121031B4E50912141612109A12E5
:1011D000171AAB0FA90E1205996026121199A312C6
:1011E00018DD1213C1401A1207DA1213C4120FF1DC
:1011F000121213121199121204A3E0D5E0DD121499
:1012000016021A3A9030071206F8120FF10206D7AA
:101210001205867B307907A3121199120580121CE2
:101220008A120FF1A3B90D004026A3E0FE20E72AA1
:10123000B420005003B40D22B4220B1212A41212D7
:10124000A7B422FA80DFB43A0C1212A2EE1212A452
:101250001212A280D01212A980CB121199A22D9243
:10126000D590017530D503122878E493A3B4FF0616
:1012700010D5EE021A3AB506F1B4B00050031212BE
:10128000A2E49320E70860061212A4A380F3120FD1
:10129000F1EE649670051212A780FB50881212A21C
:1012A000808374200218CDA3E0B40DF80218B57E37
:1012B00000572266287F01375716167F0014969034
:1012C000427F014096287580006462651080019914
:1012D00088201480005135991980014531333381BC
:1012E0000000000010FF8100000000207C000000D2
:1012F00004131213241219F21216DE121353E546C8
:10130000540162451216771213241213C1400612BB
:1013100016DE1219C71215B7901972121330121374
:10132000860213B11216DE9012E612167F021653D1
:1013300012167412134D12169812167F12169F125F
:10134000134D12167F1219F2E493B4FFEF121C7BB7
:1013500002119C1216C51216531215B7F545121636
:10136000741213DFC003894612158C1219C71216A6
:10137000A612134DD003221216771212F81216AAD3
:101380001212F202165312141A7B010215A312153F
:10139000B7F54512141A247F922A500312144B9069
:1013A00012AF121330302A091215D0121324121959
:1013B000F2E545601D0215D012167712160B1216B3
:1013C000AA021C7874FA2509B432004006F509F91E
:1013D0007B312290037E0211AF12167F12134DE46F
:1013E000FBF9A809757F31121C36C39481FC1812D1
:1013F0001C36600302145E401D0CE89405F80812C8
:101400001C36C4121C904056DC02800A121C361294
:101410001C90404ADCE874068001E4A8097A318A0D
:101420007F2840AFF509121C362212169212135370
:10143000BB002B1216C5121416121698121692E53E
:10144000467011E54560E290311EF01216921216B8
:10145000AA021653154612169F12134D80E1020A76
:10146000401215B770F81216C51216987819121C8A
:1014700036602D2480500503547F8007F404035404
:101480007FF4042480121C541216A612169F121602
:101490005312169F1219F212132712151D30D5E898
:1014A00002169F1215B770B6F54608121C3660AECC
:1014B000B48100922A400312144B1216771216922E
:1014C0001213C1502412141A2485501312167C745E
:1014D000012546500302145EF54612134D80DB9041
:1014E0001AA612167F740B80E81216C512169212F5
:1014F00019C71216A61216921219F2121653901943
:101500004D121330A312167F12134DE54612171712
:101510001219C7121386202A030215B72212169F2A
:101520001216AA121677121698021C7812167C123E
:1015300016AA12142A90311FE060E11216A61216A4
:101540009F12141A60031214A312134D12167C1268
:1015500016AA12142A75460012169212167712163F
:10156000981216A612134D0546E5461217171216C5
:101570005312167712169F1219F212151D30D5E16B
:1015800012141612169F12134D02134D12141A94B0
:1015900081500912141690050402167F9407501604
:1015A000F404FB1818121C3654F0121C54DB0122F0
:1015B000E4121C54DBEE221215D07024121C5422AB
:1015C00012141660D118121C36FF121692EF60101A
:1015D00012141A18600A121C366401121C54640199
:1015E000221213DF120586E4930217171213DF127B
:1015F0000A5DE70217171213DF8B7F121C450217D3
:10160000171213C172D550030215969016110216C7
:101610007F8500005053651213C1B380E91213C1D6
:10162000A2D580F61213C1B2D580F51213C180D6AF
:101630001213C172D580E390310C1205CAE9C313AD
:10164000F874061329C83BFA158212166E12171A7F
:1016500012160B121C7E02119C12109AD21390319A
:1016600002800B12109AD21243A884903120EAF023
:10167000A3E8F02212167712141A8027901AAC12DF
:1016800013C48B7F7B06E493121C63A319DBF7D290
:10169000242290199602167F7B31791902114F7816
:1016A000197A31021159781F80F712141A7406FA48
:1016B00028F9121C36FB121C45121C54EB121C6339
:1016C0001918DAEE2212141A7B31791F7C068A7FF0
:1016D000121C368B7F121C631217FDDCF122901A4C
:1016E000B802167F121705EB5FFAE95E802B12171E
:1016F00005EB4FFAE94E802112160B121705EB6F1E
:10170000FAE96E80141213DFAF03AE010213DF900B
:101710003100E0101801E47A00F8D224021C96E5AA
:10172000A880F4E5B880F0AA8CA88A80EDAA8DA8DC
:101730008B80E7E5B080E0E5A080DCE58880D8E537
:101740008980D4E58080D0E59080CCE58780C80290
:10175000057AE513B433F81205B9AC82AD83AB0F4B
:10176000A90E1205997015E50DB404012212181E78
:10177000AA05A8041217D1740102180DFF121B0E3E
:10178000E50D4009B40401E49F603C4022FFE50DF3
:10179000B4040122EF12181E121B07121813120EA6
:1017A000E2A904AB050EBE00010F1217F08018F479
:1017B000041205F0121813A982AB83AA0FA80E60B9
:1017C000031217D9121777AA0FA80EE50DB404015A
:1017D0002279047B30AE0D7F001218081217E51233
:1017E00018D270F52208B800010A09B900010B22CD
:1017F0001218081217FD1218D270F5002218B8FF3F
:10180000011A19B9FFF51B228B7F121C458A7F1222
:101810001C5422ECC39582FEED9583FF4E222CF9D9
:10182000E43DFB9031041205DD40F2901AD0021124
:10183000AF121A1E1210A0121B0E92D59030051274
:10184000166EA8087907C2249001758805E493FFF5
:10185000121C36FBB461004007B47B005002C2E5A5
:10186000FA121C54A3E493B502030880E320E73284
:101870006030A3E49320E70370F8A3A805B4FFCB7E
:10188000BA20030880C0302D0B202408D22412284F
:101890007802184B1218B2B422AC1218B2B422FA61
:1018A00080A4EF1218CDB4969DEB1218B51218B2A1
:1018B00080FB121C36B40D14D000D000121C63093A
:1018C0007401121C63E99404F50D790408121C6379
:1018D00009221EBEFF011FEF4E2290310A12058021
:1018E00002171A901AA012167F1216741216779009
:1018F000074D1219199031281219B7901AB21219FE
:101900001990312A1219B79012EC1213D9E9F40484
:10191000F54A7B31791302114F1213D9E9F4240FE0
:10192000F9EBF43400FB22120FC012191CC292C250
:101930008E8B8D898BC28FD28E1218D2308FFD1272
:1019400015E0D29212053A308FFD70E122800071CD
:101950003713197F0076643794800007227517804B
:101960000052359328800071918586FF810051587F
:1019700002237700449005167901082105257B0094
:10198000197355277D01701284197E003333338318
:10199000800167666616810000000010FF12115575
:1019A0001210B1740C12171712134D121653121392
:1019B000DF12191C90312402061F1218DA1205B921
:1019C000A882AA8312171A121C7502119C120525EF
:1019D000AA07EE021719A2AFC2AFC047AA48E5494D
:1019E00092AF121719D0E012171774C812171712F6
:1019F0001653121C7202119C4261642073796E743A
:101A00006178228A446976696465206279207A6502
:101A1000726F2241727261792073697A6522750A48
:101A200030750807221205257A3378001217D9126B
:101A30000691C217751333751400120D33C22DE4CD
:101A400090280293B45A031228489000FB1206E132
:101A5000D22F853E8112120DC21890305EE06434A0
:101A600070030208647D3E120755120710121831E8
:101A700020D5101217521205F92015DCD2151206C6
:101A80009180D5121A1E12103E60C590010DB4F05F
:101A900000400A121034540F1209D280B302087A9F
:101AA000880000920511850042418759810018285D
:101AB00018277C00000075838100265941319E4122
:101AC000726974682E20756E646572666C6F772219
:101AD0004D656D6F727920616C6C6F636174696FB5
:101AE0006E22A842616420617267756D656E742212
:101AF000492D737461636B2290232E30174B8542FE
:101B00000A854308020875850F83850E8222858326
:101B10000F85820E22202F27C29643870120160BA5
:101B20001021083010F412084440EFD29622A3206E
:101B30002F233013209031011206A4A30208ACA277
:101B40002F9019F88004901AF0C3853E81120D334E
:101B5000E49310E7D9121B0E40031206A01206D41C
:101B60009023BC1206E4121B071206E4302F05C2B4
:101B700020021A3A9001011206E4120FEAE4121B45
:101B80000E1205F0121BC040066004E0B401EF1213
:101B90001B07121BC0E9240AF545A31218DD121C0D
:101BA000872020CB1206D4121B0712121312120424
:101BB0007D2D121C33D545F87D5E121C33021B6F40
:101BC000AB0AA908020A91854A8CC54704B4C80823
:101BD000E40549B549020548C547D0D032121BFD7E
:101BE000C2A9C22E500A5389F0D22E43A882D28CA9
:101BF00022121BFD921E22121BFD921C221210317A
:101C00009431B32220D4FC20D3F910E7069000478A
:101C10000209D220E06E601B901C7073121C815070
:101C200063121C8D700CC083C082121C96D082D0AF
:101C300083E422020755C083C082857F838882E0C7
:101C4000D082D08322C083C082857F838982E0D006
:101C500082D08322C083C082857F838882F0D08235
:101C6000D08322C083C082857F838982F0D082D0D6
:101C70008322021CA7021C99021D6E021DA3021DD5
:101C8000E2021FCC02200B0220CE02227F02222180
:101C900002225B0222CE021FFC757F31A8091812B6
:101CA0001C36B2E0121C54121FA2EF6012BE0017C5
:101CB000121F957F06121C36121C631819DFF6E5F9
:101CC000092406F509E4229E8F308C2F50098E30AE
:101CD0008B2FF404C8C9C8FFC223BD0002D223124F
:101CE0001FBCBF0B0040027F0A752A00121EF27F44
:101CF00004792E749EC39CD4CC7001FCB450003087
:101D0000231EB3121D15500A052A7F01121EF2125E
:101D10001EA0021E8E121C3637D4F71819DFF622C9
:101D2000121C36FEE43499972ED4F71819DFF140CF
:101D300011B278792E7F04749A972400D4F719B3DE
:101D4000DFF5782B7F00E670090F0F08B82FF70238
:101D50001EE0B4100050010FE530C39F600D400B32
:101D6000F530121F2C752A00021E8E021ED9121F7A
:101D7000A2E509240CF509EEC2D59F600A4003EBE9
:101D80008001EC6001B322BD00F57F04181818191A
:101D90001919121C36FE121C459E70E60809DFF266
:101DA000D2D522121F9FBE0003021EE08D2FEF60CE
:101DB000F82E20E70610D708021ED95003021EC7CE
:101DC0009481FE121EAD7B04AC018C01121C45FAFD
:101DD000121F62EAC4121F621CDBEF8E308D2F02CD
:101DE0001E4C121FA28D2FBF0007121EC7E4D2E3A4
:101DF00022EE60B59F20E7055005021ED950BE2493
:101E000081F530121FBC7A34AB00752A007DFFD3F8
:101E10008B00792E7F045019121C36FEE434999EF3
:101E200027D4F71819DFF10D40E6E79401F7B380E6
:101E3000DF121D1577008A00A6050A7F01121F2AEE
:101E4000BA3ECAD53003021ED9752A007834E6FEA0
:101E50006004121EA018087408F928F8B60500409E
:101E600014D3E41836D4D630E40AD9F51876011222
:101E70001EA0800619E9C3C898F8792BE6C408D6D5
:101E80004206F70809B92FF4EE7003753000121FEF
:101E90009589097830E6121C631819B82AF7E422EC
:101EA0000530E53070F9D0E0D0E0021EC7C00179FE
:101EB00032121C36540FF7121C36C4540F19F7187F
:101EC00019B92AEDD00122782E7499F618B82AFB98
:101ED0007530FF121E8ED2E122121EE0E4D2E02203
:101EE000121EE9121E8ED2E222E4783DF618B829BD
:101EF000FB227C00C3EF60229402501FC000C0018F
:101F0000792E782DECD7C4FCE7D6C4F71819B92A76
:101F1000F7E7C4540FF7D001D00022FFE4C52AC56B
:101F20002BC52CC52DC52EFC80CB7C00C3EF6022B9
:101F30009402501FC000C001782A792BE6C4F6E74E
:101F4000C4D6F70809B82EF7ECC4D654F0FCD0017B
:101F5000D00022FFE4CCC52EC52DC52CC52BC52A2B
:101F600080CB540FFF783C7932E4F5331826D43017
:101F7000E403180608D68FF0E7A475F00A84C5F0CC
:101F800026D430E40205F008D618E5F019B92ADCA9
:101F90002533D4F622757F31A809740628F9221258
:101FA0001EE9121F95121C36FF121C45FE1819124D
:101FB0001C36FC121C45FB6CFD181922C000782E43
:101FC000121C45F61918B82AF7D000221220B3C007
:101FD00083C082E01223B14013121FEF400EC2E50E
:101FE000B44803D38001C3D082D08322A380E4C24B
:101FF000E5B44700400122B44100B3227B30795858
:1020000012227F740D121C63903058121EE91220A8
:10201000B31220B9927878347E7FD2D51223AE5095
:1020200008540F12208CA380F3B42E0C205169D2D7
:1020300051B834F2D25280EE20D55DB465028003EF
:10204000B445371220B21220B992501223AE504834
:10205000540FFDA31223AE500D540FCD75F00AA4FA
:102060002DFD50EF7DFFED305009C39EF404400973
:102070007401222E5003740222CE8E30B834031223
:102080001EE9E509C3940CF509021E4CC2D5700B7C
:10209000B83408305204DE0274FF22205302C252C8
:1020A0002052F32051010E2053F0B83D02D253F6D6
:1020B0000822A3E0B4201680F9B4E302800EB42B0A
:1020C000028009B4E5028003B42D02D3A322121FBB
:1020D000A2121CBFEFFE121EAD782BE517FB605855
:1020E000B4F0004003022171EE70027E80EBC45414
:1020F0000FFA1221E6CAC39AFF50087D3F12221E32
:10210000022138BA00091F12220A1222188008126E
:10211000220AEAFF1221C9EB540FFA60B01222140E
:102120001221EFB50204EA02220050FACAC39ACA89
:10213000122200EAFF0221C9EE700612221C0222BE
:10214000187BF074772E402994F7402512220D1247
:1021500021E6B408030221C91221C91221DC6068FA
:102160001222147F011221C9705E1221DC60598095
:10217000F212220D7F011221C9122214EB540F60BA
:1021800007FF1F1221C9800312216312221C7D4503
:1021900012221EEE600414B4800612221CE4800E8B
:1021A00040077D2B12221E8005122210F404C2E784
:1021B000F87A0079587B3012227F7858121C36FD4D
:1021C00012221E08E8B501F422EF600FE644300841
:1021D0001FFD12221EE4B833F0745522A900E770E7
:1021E0000409B933F922EEC394805001E4FF22C3FD
:1021F00074809E5001E422EF60FC12221C1F80F7C5
:10220000FFEF60F21222181F80F71221F7EC600C2A
:102210007D2D800A7D2E80067D3080027D20021C6F
:1022200033121FCC92231223AEB3402B7B007900D4
:102230008017A389008B021223AE400D30231812A1
:102240001FEF4003A38010240975F00A30230375A3
:10225000F01012225E50DBE492E12275F00AC0E039
:10226000C0F0E9A4F9EBABF0D0F0A4A2D292D52B48
:10227000FBD0E072D54007540F29F9E43BFB22E480
:102280009027101222A19003E81222A1900064125C
:1022900022A190000A1222A19000011222A1602026
:1022A000227EFF0ECAB58300CA4012C89582C8CAF2
:1022B0009583CA50EEC82582C8CA3583CA4E60E0ED
:1022C00074302E8B7F121C6309B900010B2212227D
:1022D0001CA2369223EB1222F7EB1222F8C223E95A
:1022E0001222F7E91222F87D4802221EC22324900E
:1022F000D43440D4FD80F2C4540F70F03023ED226A
:10230000201A0302281B0228884E6F206461746122
:10231000229441726974682E206F766572666C6FC4
:10232000772250726F6772616D6D696E67224361CB
:102330006E277420636F6E74696E756522496E76C0
:10234000616C6964206C696E65206E756D62657282
:102350002250524F4D206D6F6465220D0A0A44537E
:102360003530303020546F7073696465204261737A
:10237000696320496E746572707265746572205667
:10238000322E30312032302D4D61792D31393936B0
:102390002032333A30302057495448203130322EE1
:1023A00041534D20455854454E53494F4E2212201B
:1023B000B3B43A00400122B43000B3224572726FC8
:0423C000723A20222B
:00000001FF
